:020000040000FA
:020000001028C6
:08000800A0000308A10021087B
:080010008300A00E200E090080
:10002000FF23831690008F3081009F019601990174
:100030008B0183129F010730990085010A30CC2281
:100040008316C8308500831285140230D2228510B1
:1000500085191E28C1210A30CC224C28E4210A30FF
:10006000CC221D210A30CC2280210A30CC225A21F8
:100070000A30CC22F2210A30CC2245210A30CC228F
:10008000D3210A30CC229521E4219521AC210A30DC
:10009000CC22C121D321AC218316C8308500831224
:1000A00085140530CC2285107D220A30CC22051023
:1000B0001430D22283220F30CC2205101430D222E9
:1000C0007D220A30CC2205100530CC228316C830A0
:1000D0008500831264009E018C221E08B500E02278
:1000E0000A30CC225C2258220A30CC220A30CC22A0
:1000F00085140230D2228510851976288316C830DF
:1001000085008312C1210A30B800B901B90A7D22E5
:1001100085140230D22285106430D222783039061C
:100120000319CD288519862805100130CC22F62028
:10013000B803B901380838050319A52883220F3000
:10014000CC2205101430D22286281D210510023041
:10015000CC221D2183220330CC220510F2217D22E6
:100160000330CC22051083220430CC220510F2216A
:100170007D220530CC2205101D2183220330CC22A4
:100180000510F2217D220330CC2283220330CC22C1
:100190000510D321C830CC227E2805100230CC2295
:1001A00080210A30CC228322C1210430CC22D321E9
:1001B0000430CC229521AC219521C1210430CC22E0
:1001C000D3210430CC2205106430CC229521E421C7
:1001D0009521AC217E280A30B600C3226300851D1C
:1001E000F328B60BEE288519F528000008303802F0
:1001F0000318080038083907BA000F30BA05BA0BDF
:1002000002294529BA0B05291D29BA0B0829D3292A
:10021000BA0B0B29E429BA0B0E291D29BA0B112997
:100220005A29BA0B14298029BA0B17290800BA0BCE
:100230001A299529BA0BFF28AC2925210730D2228B
:1002400025210730D222252108003C30B100413061
:10025000A9002908AB008316051285128312051622
:100260008512303085060B30A2000000000000002F
:100270006400A20B3529AB0B31290630D822A90323
:10028000B10B29290512851208007830A8000F301B
:10029000A9001430AA0000220130CC22B430A800FA
:1002A0000F30A9001830AA0020223230A9002B08F4
:1002B000602208005030A8000F30A9002230AA00A8
:1002C0002022B430A9002B0860220130CC226430F7
:1002D000A8000F30A9001E30AA0020227830A90003
:1002E0002B0860220130CC22C830A8000F30A900B2
:1002F0001E30AA0020225030A9002B0860220800DE
:10030000B430A8000F30A9001830AA002022013014
:10031000CC226430A8001930A9001430AA000022B1
:100320005030A9002B08602208000830AF0032309E
:10033000A8000F30A9001430AA0000221430AF0B1F
:1003400097290830AF004630A8000C30A9000022E1
:100350001430AF0BA32908000830AF003230A800DA
:100360000F30A90020221430AF0BAE290B30AF00A4
:100370004630A8000C30A90020221430AF0BB82959
:1003800008001E30B0001E30A8000F30A9000F304A
:10039000AA000230AF0020226400AF0BCB29A803D3
:1003A000B00BC92908001E30B0000A30A8000C307C
:1003B000A9000230AF0020226400AF0BDB29A80A9D
:1003C000A80AB00BD92908001430AF001930A800D2
:1003D0000F30A9000A30AA0000220A30D222AF0B47
:1003E000E62908000730AF003230A8003730A900F6
:1003F0000530AA0000226430D222AF0BF429080095
:1004000083160508B700051285128312051685129A
:100410002808AB002908AC002A08AD002B08A20070
:10042000A20B102A30308506AD0B0E2AAB03AC0BA5
:100430000C2A0512851283163708850083120800DE
:1004400083160508B700051285128312051685125A
:100450002808AB002908AC002A08AD002B08A20030
:10046000A20B302A30308506AD0B2E2AAB0AAC0B1E
:100470002C2A05128512831637088500831208007E
:10048000A800B430A7008316051285128312051642
:1004900085122808D82230308506A70B492A080083
:1004A0003230A900ED30602A6530A9007530602A2D
:1004B000BE30A9001D30602AE230A9001830602A41
:1004C0006400A80083160508B70005128512831280
:1004D000051685120830AE002808A200A20B6E2A6D
:1004E00030308506AE0B6C2AA90B6A2A05128512DC
:1004F0008316370885008312080005100A30D222BF
:1005000005150514080005100A30D222051105143E
:1005100008000515051008008316FD3085005830C9
:100520009F00831285140D309F000530CC229F144C
:100530003C30D2221430D8229F189A2A8510080005
:1005400083169E01FD30850050309F008312851078
:100550003C30D2228316FF30850083121430CC2227
:10056000831652309F00831285309F000230D222C2
:100570009F143C30D2221430D8229F18BB2A8316F5
:100580001E088312080007309900850183169F0119
:10059000FF30850083120800A5002830D222A50B69
:1005A000CD2A0800A300FA30D822A30BD32A0800D2
:1005B000A200DE226400A203220FD92A0800B5009F
:1005C000B301B40164303502031CE92AB500B30A53
:1005D000E22A0A303502031CF02AB500B40AE92ADF
:1005E000FE220A30CC223408B300FE220A30CC228C
:1005F0003508B300FE220530CC220800B308031DE5
:10060000032B502200340130B302031C0034542267
:060610000530CC22032B93
:0C07B400203428346334293432343034CB
:1007C0003034373420344134703470346C3469340C
:1007D00065346434203449346E347334703469348D
:1007E00072346134743469346F346E3473342C343D
:0A07F00020344C344C3443342034E0
:02400E008C3FE5
:00000001FF
